:02000000017B82
:20007B0075810E905CE979007A007B6E7C18EB4C601CE493A3CAC583CAC9C582C9F0A3CA3D
:20009B00C583CAC9C582C91BBBFFE31C80E0901896E4F01249EC12001B80FBC82581C822CD
:2000BB00C92581C97A0022D083D082CF2581F581CFC082C08322CF2581F581CF22FBE0CBC9
:2000DB0022FCE0FBA3E0CC22FAE0F9A3E0CA2229F9E5F03AFA227C00CB30E7011CCB22752F
:2000FB00F00030E70215F022FDE493A3FEE493A3FF4E7009E493FE740193FF800BE493A39F
:20011B00B5050BE493B5F0068F838E82E473A380D8FEEBA4FD8EF0ECA4FCEB8EF0A4C5F013
:20013B002C2DC5F02231468EF0ED22C002C001AAF0F97E007D007F11C3E933F9EA33FADF01
:20015B0008F5F0E9D001D00222ED33FDEE33FEC3ED9BF5F0EE9C40E0ADF0FED380DBBB004F
:20017B000122C333C5F033C5F0DBF722BB000122C3C5F013C5F013DBF722240280022401C8
:20019B00C5F03400C5F022C394028003C39401C5F09400C5F02231A7F4C5F0F4C5F022459F
:2001BB00F07022042251094024801A5109401E7014801A5109400E7014800A5109500E8060
:2001DB0004511D6008E4F5F022511D60F8E4F5F00422511D40F780ED511D40F170E780ED15
:2001FB00511D40E170E780DD511D50E180D7C39BC5F09C20E70720D207C345F02220D2F9F0
:20021B00D322C5F0C39C7003E5F09B22901896E0A360EEE0FFA3E0A3CF2582F582EF35830D
:20023B00F58380EB5388CC5389F0438901758A66758CFCE4F5F022D2A9D2B9D2AF438810D1
:20025B00E4F5F022C2A95388EFE4F5F022C2AFE4F5F0F50885F009E4F5F0F50A85F00BE497
:20027B00F5F0901872F0A3C5F0F0C5F0D2AFE4F5F02205810581E5088509F078F91200B65B
:20029B0026C5F00836C5F0080808F608A6F0E5088509F078FD1200B686030886041201ED06
:2002BB0060030202A978FD1200B6E60886F01581158122C2AFC0D0C0E0C0F0C083C082C08E
:2002DB0000C001C002C003C004C005C006C0075388EF758A66758CFC438810E5088509F035
:2002FB00120199F50885F0091201A7E50A850BF0120199F50A85F00B1201A7E50A850BF03F
:20031B007BF47C011201DC70030203A3E4F5F0F50A85F00B90188BE00490188BF01490188E
:20033B008BE075F0007B027C0012014090188BF0901876E090188B1200D84B90188AF0E4F7
:20035B0075F0C0C0E0C0F090188AE075F000C0E0C0F012599A158115811581158190188BB6
:20037B00E070030203A3E4F5F0F50A85F00B901872E0A3F5F0E0C5F0120199901872F0A3AF
:20039B00C5F0F0C5F01201A743871075FF01B29790186EE590F090186FE5B0F0901870E582
:2003BB00C0F0901871E5C4F0D007D006D005D004D003D002D001D000D082D083D0F0D0E00F
:0603DB00D0D0D2AF3222A7
:03000B000202CE20
:2003E20022C29590A0087400F0740275F000C0E0C0F012028D1581158190A00074BCC29636
:20040200F0D29690A0017482C296F0D29690A002741EC296F0D29690A0047400C296F0D275
:2004220096741B75F000C0E0C0F01259BA15811581740075F007C0E0C0F01259DA1581156F
:2004420081741B75F000C0E0C0F01259BA15811581740775F007C0E0C0F01259DA1581155D
:2004620081740A75F007C0E0C0F01259DA1581158122C29590A0087400F0740275F000C09E
:20048200E0C0F012028D1581158190A00074BCC296F0D29690A0017461C296F0D29690A007
:2004A20002741EC296F0D29690A0047400C296F0D29622C29590A0087400F0740275F000AE
:2004C200C0E0C0F012028D1581158190A00074BCC296F0D29690A0017482C296F0D2969086
:2004E200A002741EC296F0D29690A0047400C296F0D29622C29590A0087400F0740275F0CE
:2005020000C0E0C0F012028D1581158190A00074BCC296F0D29690A00174A3C296F0D296B4
:2005220090A002741EC296F0D29690A0047400C296F0D296220581058178F91200B6E6752B
:20054200F00008080808F608A6F0741B75F000C0E0C0F01259BA15811581741A75F007C0A6
:20056200E0C0F01259DA15811581741B75F000C0E0C0F01259BA15811581742175F007C022
:20058200E0C0F01259DA15811581742475F007C0E0C0F078F51200B6E675F000C0E0C0F034
:2005A200740212584E1581158115811581C295741275F000C0E0C0F012028D1581158178DC
:2005C200F71200B6E675F0007BFF7C0012012C7B647C0012014678FD1200B6F608A6F0183D
:2005E200E60886F0F50C90A0007411C296F0D29690A0017421C296F0D29690A002E50CC2D4
:2006020096F0D29690A0037400C296F0D29690A0087455F0D295741275F000C0E0C0F012EE
:20062200028D1581158115811581220581058178F91200B6E675F00008080808F608A6F06B
:20064200741B75F000C0E0C0F01259BA15811581743475F007C0E0C0F01259DA158115812E
:20066200741B75F000C0E0C0F01259BA15811581743B75F007C0E0C0F01259DA1581158107
:20068200743E75F007C0E0C0F078F51200B6E675F000C0E0C0F0740212584E1581158115AB
:2006A200811581C295741275F000C0E0C0F012028D1581158178F71200B6E675F0007BFFC6
:2006C2007C0012012C7B647C0012014678FD1200B6F608A6F018E60886F0F50C90A00074B7
:2006E20044C296F0D29690A0017424C296F0D29690A002E50CC296F0D29690A0037400C24F
:2007020096F0D29690A0087455F0D295741275F000C0E0C0F012028D15811581158115815D
:20072200220581058178F71200B6E675F00078FD1200B6F608A6F0741B75F000C0E0C0F0F2
:200742001259BA15811581744E75F007C0E0C0F01259DA15811581741B75F000C0E0C0F013
:200762001259BA15811581745575F007C0E0C0F01259DA15811581745875F007C0E0C0F0A8
:2007820078F31200B6E675F000C0E0C0F0740212584E1581158115811581C295740675F0CD
:2007A20000C0E0C0F012028D1581158178F51200B6E675F0007BFF7C0012012C7B647C000A
:2007C20012014678FD1200B6F608A6F018E60886F0F50C78F91200B6E675F0007B007C00F5
:2007E2001201DC700302081590A00074CCC296F0D29690A001742CC296F0D29690A002E5BE
:200802000CC296F0D29690A0037400C296F0D29602083D90A0007485C296F0D29690A00172
:20082200746BC296F0D29690A002E50CC296F0D29690A0037400C296F0D29690A0087455FC
:20084200F0D295741275F000C0E0C0F012028D1581158115811581220581058105810581D1
:20086200E4F5F078FB1200B6F608A6F0D294D293901876E054FB901876F054F7901876F05F
:20088200547F901876F04402901876F0E475F0C0C0E0C0F0901876E075F000C0E0C0F01203
:2008A200599A1581158115811581901888E075F000C0E0C0F0121E6415811581901882E05C
:2008C200A3F5F0E0C5F078FD1200B6F608A6F012026890187FE075F000C0E0C0F0741575F2
:2008E200F000C0E0C0F0901880E075F000C0E0C0F01207237FFA1200C278FB1200B6E60847
:2009020086F045F06003020B1090186EE0540175F00045F0700690186EE054026003020995
:2009220056740275F000C0E0C0F012028D1581158190186EE0540175F00045F07006901864
:200942006EE054026003020956E4F50E74F175F0FF020BD490186EE0540175F00045F07047
:200962000690186EE0540275F00045F0600C901871E054081200FA1201BA45F0700302093C
:20098200CB740275F000C0E0C0F012028D1581158190186EE0540175F00045F0700690188F
:2009A2006EE0540275F00045F0600C901871E054081200FA1201BA45F070030209CBE4F506
:2009C2000E74F075F0FF020BD4E5088509F078FD1200B686030886041201FB7003020B0D00
:2009E20090186EE054046003020A16740275F000C0E0C0F012028D1581158190186EE054E0
:200A0200046003020A16740175F00078FB1200B6F608A6F090186FE054047003020B0D7452
:200A22000275F000C0E0C0F012028D1581158190186FE054047003020B0D1202681203E3E0
:200A4200D294D293901876E054FD901876F054FB901876F054F7901876F04440901876F024
:200A6200E475F0C0C0E0C0F0901876E075F000C0E0C0F012599A158115811581158174692E
:200A820075F007C0E0C0F01259DA15811581E4F5F0901874F0A3C5F0F0C5F0901872E0A3B8
:200AA200F5F0E0C5F07B3C7C001201ED7003020AF2901872E0A3F5F0E0C5F09018741200D1
:200AC200DC1201FB7003020AEF742E75F000C0E0C0F01259BA15811581901872E0A3F5F092
:200AE200E0C5F0901874F0A3C5F0F0C5F0020A9D747575F007C0E0C0F01259DA1581158197
:200B0200121C7574F375F0FF020BD40208FB901870E054801200FA1201BA45F06003020B35
:200B220076740275F000C0E0C0F012028D15811581901870E054801200FA1201BA45F0600B
:200B420003020B76901876E04480901876F0E475F0C0C0E0C0F0901876E075F000C0E0C021
:200B6200F012599A158115811581158174F375F0FF020BD4C294D293901876E054FD9018C8
:200B820076F054FB901876F04408901876F0E475F0C0C0E0C0F0901876E075F000C0E0C01A
:200BA200F012599A1581158115811581901881E075F000C0E0C0F0741475F000C0E0C0F0EB
:200BC200E4C0E0C0F01207237FFA1200C2740175F000158115811581158122901881E07584
:200BE200F000C0E0C0F0741475F000C0E0C0F0E4C0E0C0F01207237FFA1200C2C294D293FE
:200C0200901876E054FD901876F054FB901876F04408901876F0E475F0C0C0E0C0F09018BD
:200C220076E075F000C0E0C0F012599A1581158115811581220581058105810581E4F5F047
:200C420078FB1200B6F608A6F0D294D293901876E054FB901876F054F7901876F0547F90E1
:200C62001876F04402901876F0E475F0C0C0E0C0F0901876E075F000C0E0C0F012599A157A
:200C820081158115811581901887E075F000C0E0C0F0121E641581158190187AE0A3F5F001
:200CA200E0C5F078FD1200B6F608A6F0120268901877E075F000C0E0C0F0741575F000C0EE
:200CC200E0C0F012062D158115811581158178FB1200B6E60886F045F06003020E569018A0
:200CE2006EE054016003020D11740275F000C0E0C0F012028D1581158190186EE054016029
:200D020003020D11E4F50D74F275F0FF020EC8E5088509F078FD1200B68603088604120150
:200D2200FB7003020D5C90186EE054046003020D5C740275F000C0E0C0F012028D15811545
:200D42008190186EE054046003020D5C740175F00078FB1200B6F608A6F090186FE05404FC
:200D62007003020E53740275F000C0E0C0F012028D1581158190186FE054047003020E537E
:200D82001202681203E3D294D293901876E054FD901876F054FB901876F054F7901876F0FF
:200DA2004440901876F0E475F0C0C0E0C0F0901876E075F000C0E0C0F012599A1581158162
:200DC20015811581748575F007C0E0C0F01259DA15811581E4F5F0901874F0A3C5F0F0C5DD
:200DE200F0901872E0A3F5F0E0C5F07B3C7C001201ED7003020E38901872E0A3F5F0E0C5D5
:200E0200F09018741200DC1201FB7003020E35742E75F000C0E0C0F01259BA1581158190D8
:200E22001872E0A3F5F0E0C5F0901874F0A3C5F0F0C5F0020DE3749175F007C0E0C0F0125B
:200E420059DA15811581121C7574F375F0FF020EC8020CD0901870E054801200FA1201BA68
:200E620045F06003020EBC740275F000C0E0C0F012028D15811581901870E054801200FA3C
:200E82001201BA45F06003020EBC901876E04480901876F0E475F0C0C0E0C0F0901876E0F8
:200EA20075F000C0E0C0F012599A158115811581158174F375F0FF020EC8120ED178FB1205
:200EC20000B6E60886F0158115811581158122901879E075F000C0E0C0F0741475F000C019
:200EE200E0C0F012062D158115811581158190186EE0540275F00045F06006901871E0542A
:200F0200087003020F0DC294020F11C293D294901876E054FD901876F054F7901876F04409
:200F220004901876F0E475F0C0C0E0C0F0901876E075F000C0E0C0F012599A15811581154B
:200F420081158122D293D294901876E054FD901876F054F7901876F054FB901876F0547FA5
:200F6200901876F0E475F0C0C0E0C0F0901876E075F000C0E0C0F012599A1581158115818E
:200F820015811203E3740275F000C0E0C0F012028D15811581220581058105810581E4F5B6
:200FA200F078FB1200B6F608A6F0901876E054FB901876F054F7901876F0547F901876F0DB
:200FC2004402901876F0E475F0C0C0E0C0F0901876E075F000C0E0C0F012599A158115817E
:200FE20015811581C293D29490186EE0540275F00045F06006901871E054087003021006DC
:20100200D293C294901887E075F000C0E0C0F0121E641581158174C875F00078FD1200B6B1
:20102200F608A6F0120268901877E075F000C0E0C0F0741575F000C0E0C0F012062D1581D1
:2010420015811581158178FB1200B6E60886F045F060030211B090186FE0540470030211FD
:201062004F740275F000C0E0C0F012028D1581158190186FE05404700302114F1202681275
:2010820003E3D294D293901876E054FD901876F054FB901876F054F7901876F0444090185E
:2010A20076F0E475F0C0C0E0C0F0901876E075F000C0E0C0F012599A15811581158115815F
:2010C20074A175F007C0E0C0F01259DA15811581E4F5F0901874F0A3C5F0F0C5F0901872E0
:2010E200E0A3F5F0E0C5F07B3C7C001201ED7003021134901872E0A3F5F0E0C5F0901874D1
:201102001200DC1201FB7003021131742E75F000C0E0C0F01259BA15811581901872E0A3D5
:20112200F5F0E0C5F0901874F0A3C5F0F0C5F00210DF74AD75F007C0E0C0F01259DA158181
:201142001581121C7574F375F0FF02138F90186EE05402600302118A740275F000C0E0C05E
:20116200F012028D1581158190186EE0540175F00045F0700690186EE05402600302118A09
:2011820074F275F0FF02138FE5088509F078FD1200B686030886041201FB70030211AD7467
:2011A2000175F000181818F608A6F0021048901876E054FD901876F054F7901876F0440493
:2011C200901876F0E475F0C0C0E0C0F0901876E075F000C0E0C0F012599A1581158115812C
:2011E2001581901879E075F000C0E0C0F0741575F000C0E0C0F012062D1581158115811547
:2012020081120268745875F00278FD1200B6F608A6F0E4F5F0181818F608A6F078FB1200A1
:20122200B6E60886F045F0600302138690186FE054047003021325740275F000C0E0C0F038
:2012420012028D1581158190186FE0540470030213251202681203E3D294D293901876E086
:2012620054FD901876F054FB901876F054F7901876F04440901876F0E475F0C0C0E0C0F06C
:20128200901876E075F000C0E0C0F012599A158115811581158174BD75F007C0E0C0F0123D
:2012A20059DA15811581E4F5F0901874F0A3C5F0F0C5F0901872E0A3F5F0E0C5F07B3C7CB1
:2012C200001201ED700302130A901872E0A3F5F0E0C5F09018741200DC1201FB70030213C3
:2012E20007742E75F000C0E0C0F01259BA15811581901872E0A3F5F0E0C5F0901874F0A377
:20130200C5F0F0C5F00212B574C975F007C0E0C0F01259DA15811581121C7574F375F0FFD0
:2013220002138F90186EE054026003021360740275F000C0E0C0F012028D15811581901843
:201342006EE0540175F00045F0700690186EE05402600302136074F275F0FF02138FE50859
:201362008509F078FD1200B686030886041201FB7003021383740175F000181818F608A6B6
:20138200F002121E78FB1200B6E60886F01581158115811581220581058105810581E4F51F
:2013A200F078FB1200B6F608A6F0901888E075F000C0E0C0F0121E6415811581901882E0DD
:2013C200A3F5F0E0C5F07B037C0012012C7B047C0012014678FD1200B6F608A6F012026814
:2013E20090187FE075F000C0E0C0F0741575F000C0E0C0F0901880E075F000C0E0C0F01222
:2014020007237FFA1200C2D294D293901876E04404901876F054F7901876F0547F901876EA
:20142200F04402901876F0E475F0C0C0E0C0F0901876E075F000C0E0C0F012599A158115AA
:20144200811581158190186EE054016003021475740275F000C0E0C0F012028D15811581AC
:2014620090186EE05401600302147574F175F0FF02168E90186EE0540175F00045F0600C71
:20148200901871E054081200FA1201BA45F070030214CD740275F000C0E0C0F012028D15B0
:2014A20081158190186EE0540175F00045F0600C901871E054081200FA1201BA45F07003EC
:2014C2000214CD74F075F0FF02168EE5088509F078FD1200B686030886041201FB70030273
:2014E200160F90186EE054046003021518740275F000C0E0C0F012028D1581158190186ED7
:20150200E054046003021518740175F00078FB1200B6F608A6F090186FE05404700302167C
:201522000F740275F000C0E0C0F012028D1581158190186FE05404700302160F120268122B
:2015420003E3D294D293901876E054FD901876F054FB901876F054F7901876F04440901899
:2015620076F0E475F0C0C0E0C0F0901876E075F000C0E0C0F012599A15811581158115819A
:2015820074D975F007C0E0C0F01259DA15811581E4F5F0901874F0A3C5F0F0C5F0901872E3
:2015A200E0A3F5F0E0C5F07B3C7C001201ED70030215F4901872E0A3F5F0E0C5F090187448
:2015C2001200DC1201FB70030215F1742E75F000C0E0C0F01259BA15811581901872E0A34D
:2015E200F5F0E0C5F0901874F0A3C5F0F0C5F002159F74E575F007C0E0C0F01259DA1581C0
:201602001581121C7574F375F0FF02168E78FB1200B6E60886F045F0700302144790187062
:20162200E054801200FA1201BA45F06003021685740275F000C0E0C0F012028D15811581EE
:20164200901870E054801200FA1201BA45F06003021685901876E04480901876F0E475F095
:20166200C0C0E0C0F0901876E075F000C0E0C0F012599A158115811581158174F375F0FF7D
:2016820002168E78FB1200B6E60886F0158115811581158122058105810581120268D29415
:2016A200C293E5088509F078F81200B686030886041201ED700302188790186EE054027045
:2016C200030216ED740275F000C0E0C0F012028D1581158190186EE0540270030216ED74D0
:2016E20001F50E74F475F0FF021A6290186EE0540175F00045F06006901871E05408700387
:2017020002173D740275F000C0E0C0F012028D1581158190186EE0540175F00045F060062E
:20172200901871E05408700302173DC294D2937401F50E74F675F0FF021A6290186FE054BF
:20174200047003021834740275F000C0E0C0F012028D1581158190186FE0540470030218EE
:20176200341202681203E3D294D293901876E054FD901876F054FB901876F054F7901876D1
:20178200F04440901876F0E475F0C0C0E0C0F0901876E075F000C0E0C0F012599A15811509
:2017A200811581158174F575F007C0E0C0F01259DA15811581E4F5F0901874F0A3C5F0F0C7
:2017C200C5F0901872E0A3F5F0E0C5F07B3C7C001201ED7003021819901872E0A3F5F0E000
:2017E200C5F09018741200DC1201FB7003021816742E75F000C0E0C0F01259BA15811581CF
:20180200901872E0A3F5F0E0C5F0901874F0A3C5F0F0C5F00217C4740175F008C0E0C0F097
:201822001259DA15811581121C7574F375F0FF021A6290186EE0540175F00045F0600C9068
:201842001871E054081200FA1201BA45F07003021884740275F000C0E0C0F012028D158140
:20186200158190186EE0540175F00045F0600C901871E054081200FA1201BA45F0600302B7
:2018820018870216A4D294C293E4F50E1203E3901887E075F000C0E0C0F0121E641581154E
:2018A20081901884E078FE1200B6F6901885E0A3F5F0E0C5F01818F608A6F012026878FE85
:2018C2001200B6E675F000C0E0C0F07415C0E0C0F012062D1581158115811581E5088509B2
:2018E200F078FC1200B686030886041201ED7003021A5A901871E0540875F00045F0600661
:2019020090186EE05401700302191574F675F0FF021A6290186FE0540470030219F11202A9
:20192200681203E3D294D293901876E054FD901876F054FB901876F054F7901876F04440E3
:20194200901876F0E475F0C0C0E0C0F0901876E075F000C0E0C0F012599A158115811581A4
:201962001581741175F008C0E0C0F01259DA15811581E4F5F0901874F0A3C5F0F0C5F090BA
:201982001872E0A3F5F0E0C5F07B3C7C001201ED70030219D6901872E0A3F5F0E0C5F09080
:2019A20018741200DC1201FB70030219D3742E75F000C0E0C0F01259BA158115819018727A
:2019C200E0A3F5F0E0C5F0901874F0A3C5F0F0C5F0021981741D75F008C0E0C0F01259DAD0
:2019E20015811581121C7574F375F0FF021A62901870E054801200FA1201BA45F06003028E
:201A02001A57740275F000C0E0C0F012028D15811581901870E054801200FA1201BA45F081
:201A22006003021A57901876E04480901876F0E475F0C0C0E0C0F0901876E075F000C0E0A2
:201A4200C0F012599A158115811581158174F375F0FF021A620218DE120ED1740175F0006B
:201A620015811581158122058105810581120268E5088509F078F81200B6860308860412A2
:201A820001ED7003021AEB90186EE0540175F00045F0600C901871E054081200FA1201BA5D
:201AA20045F07003021AB174F575F0FF021C6E90186EE054027003021AC474F475F0FF02E9
:201AC2001C6E90186EE0540175F00045F06006901871E054087003021AE87401F50E74F681
:201AE20075F0FF021C6E021A72E4F50D901889E07003021B06D293D2941203E3740175F03C
:201B020000021C6E90187CE078FE1200B6F690187DE0A3F5F0E0C5F01818F608A6F0120205
:201B22006878FE1200B6E675F000C0E0C0F07414C0E0C0F01205371581158115811581D212
:201B420093D294E5088509F078FC1200B686030886041201ED7003021C6690186EE0540186
:201B62007003021B721203E374EF75F0FF021C6E90186EE054027003021B87C29374F47581
:201B8200F0FF021C6E90186FE054047003021C631202681203E3D294D293901876E054FDF7
:201BA200901876F054FB901876F054F7901876F04440901876F0E475F0C0C0E0C0F09018CC
:201BC20076E075F000C0E0C0F012599A1581158115811581742D75F008C0E0C0F01259DAF8
:201BE20015811581E4F5F0901874F0A3C5F0F0C5F0901872E0A3F5F0E0C5F07B3C7C001289
:201C020001ED7003021C48901872E0A3F5F0E0C5F09018741200DC1201FB7003021C457482
:201C22002E75F000C0E0C0F01259BA15811581901872E0A3F5F0E0C5F0901874F0A3C5F0F3
:201C4200F0C5F0021BF3743975F008C0E0C0F01259DA15811581121C7574F375F0FF021C66
:201C62006E021B451203E3740175F000158115811581220581D293D294901876E054FD90AC
:201C82001876F054F7901876F054FB901876F04480901876F0E475F0C0C0E0C0F0901876C5
:201CA200E075F000C0E0C0F012599A15811581158115811202681203E3901870E0548012DE
:201CC20000FA1201BA45F06003021D6B90186EE0540175F00045F0700690186EE054027002
:201CE20003021D43E5088509F07B647C001201FB7003021D4012026878FE1200B6E606E64B
:201D020075F0007B027C00120140F675F0007B077C001201799018761200D84B90188AF0B6
:201D2200E475F0C0C0E0C0F090188AE075F000C0E0C0F012599A1581158115811581021C06
:201D4200CE901876E04480901876F0E475F0C0C0E0C0F0901876E075F000C0E0C0F012596C
:201D62009A15811581158115811581220581D293D294901876E054FD901876F054F7901816
:201D820076F054FB901876F0547F901876F0E475F0C0C0E0C0F0901876E075F000C0E0C081
:201DA200F012599A15811581158115811203E3901870E054801200FA1201BA45F06003029D
:201DC2001E6190186EE0540175F00045F0700690186EE054027003021E39E5088509F07B29
:201DE200647C001201FB7003021E3612026878FE1200B6E606E675F0007B027C00120140ED
:201E0200F675F0007B077C001201799018761200D84B90188AF0E475F0C0C0E0C0F0901865
:201E22008AE075F000C0E0C0F012599A1581158115811581021DC4901876E0448090187661
:201E4200F0E475F0C0C0E0C0F0901876E075F000C0E0C0F012599A15811581158115811512
:201E62008122C295743275F000C0E0C0F012028D1581158178FB1200B6E620E003021E8773
:201E8200C2C0021E89D2C078FB1200B6E620E103021E9AC2C1021E9CD2C178FB1200B6E6B1
:201EA20020E203021EADC2C2021EAFD2C278FB1200B6E620E303021EC0C2C3021EC2D2C364
:201EC20078FB1200B6E620E403021ED3C2C4021ED5D2C4741475F000C0E0C0F012028D15E1
:201EE200811581227F061200C278F51200B6E60886F07B017C001201DC7003021F40E475A1
:201F0200F0C0C0E0C0F01259791581158178F91200B6F608A6F018E60886F05440C5F054C9
:201F220000C5F01201BA901889F0D2C5D2C6741475F000C0E0C0F012028D1581158178F556
:201F42001200B6E60886F07B027C001201DC7003021F95E475F0D0C0E0C0F012597915815F
:201F6200158178F91200B6F608A6F018E60886F05440C5F05400C5F01201BA901889F0C27E
:201F8200C5D2C6741475F000C0E0C0F012028D1581158178F51200B6E60886F07B037C0045
:201FA2001201DC7003021FEAE475F0E0C0E0C0F01259791581158178F91200B6F608A6F05C
:201FC20018E60886F05440C5F05400C5F01201BA901889F0C2C5C2C6741475F000C0E0C0E7
:201FE200F012028D1581158178F91200B6E60886F054BFC5F05400C5F018F608A6F018E60A
:202002000886F07B0E7C0012012C08F608A6F018E60886F012019918F608A6F01201A7C30F
:2020220033C5F033C5F079007A001200EA89828A83E0A3F5F0E0C5F078FD1200B6F608A6E9
:20204200F018E60886F0901877F0181818E60886F012019918F608A6F01201A7C333C5F09A
:2020620033C5F079007A001200EA89828A83E0A3F5F0E0C5F078FD1200B6F608A6F018E6A3
:202082000886F0901878F0181818E60886F012019918F608A6F01201A7C333C5F033C5F05F
:2020A20079007A001200EA89828A83E0A3F5F0E0C5F078FD1200B6F608A6F012586E5440DD
:2020C200C5F05400C5F07B067C0012018745F0700302211E12586E5480C5F05400C5F07BDB
:2020E200077C0012018745F0700302210878FD1200B6E60886F02406C5F03400C5F018F677
:2021020008A6F002211E78FD1200B6E60886F02403C5F03400C5F018F608A6F012586E54A0
:2021220040C5F05400C5F07B067C0012018745F0600302216712586E5480C5F05400C5F07C
:202142007B077C0012018745F0700302216778FD1200B6E60886F0C39403C5F09400C5F0BA
:2021620018F608A6F078FD1200B6E60886F0901879F0181818E60886F012019918F608A6EB
:20218200F01201A7C333C5F033C5F079007A001200EA89828A83E0A3F5F0E0C5F090187ADA
:2021A200F0A3C5F0F0C5F078FB1200B6E60886F012019918F608A6F01201A7C333C5F033A1
:2021C200C5F079007A001200EA89828A83E0A3F5F0E0C5F078FD1200B6F608A6F018E6086D
:2021E20086F090187CF0181818E60886F012019918F608A6F01201A7C333C5F033C5F07989
:20220200007A001200EA89828A83E0A3F5F0E0C5F090187DF0A3C5F0F0C5F078FB1200B6E4
:20222200E60886F012019918F608A6F01201A7C333C5F033C5F079007A001200EA89828A0F
:2022420083E0A3F5F0E0C5F078FD1200B6F608A6F018E60886F090187FF0181818E60886DC
:20226200F012019918F608A6F01201A7C333C5F033C5F079007A001200EA89828A83E0A33D
:20228200F5F0E0C5F078FD1200B6F608A6F018E60886F0901880F0181818E60886F012019E
:2022A2009918F608A6F01201A7C333C5F033C5F079007A001200EA89828A83E0A3F5F0E03B
:2022C200C5F078FD1200B6F608A6F012586E5440C5F05400C5F07B067C0012018745F07010
:2022E2000302232E12586E5480C5F05400C5F07B077C0012018745F0700302231878FD1218
:2023020000B6E60886F02406C5F03400C5F018F608A6F002232E78FD1200B6E60886F02415
:2023220003C5F03400C5F018F608A6F012586E5440C5F05400C5F07B067C0012018745F058
:20234200600302237712586E5480C5F05400C5F07B077C0012018745F0700302237778FDC1
:202362001200B6E60886F0C39403C5F09400C5F018F608A6F078FD1200B6E60886F09018E2
:2023820081F0181818E60886F012019918F608A6F01201A7C333C5F033C5F079007A001274
:2023A20000EA89828A83E0A3F5F0E0C5F0901882F0A3C5F0F0C5F078FB1200B6E60886F066
:2023C20012019918F608A6F01201A7C333C5F033C5F079007A001200EA89828A83E0A3F5D7
:2023E200F0E0C5F078FD1200B6F608A6F018E60886F0901884F0181818E60886F012019995
:2024020018F608A6F01201A7C333C5F033C5F079007A001200EA89828A83E0A3F5F0E0C5AD
:20242200F0901885F0A3C5F0F0C5F078FB1200B6E60886F012019918F608A6F01201A7C31C
:2024420033C5F033C5F079007A001200EA89828A83E0A3F5F0E0C5F078FD1200B6F608A6C5
:20246200F018E60886F0901887F0181818E60886F012019918F608A6F01201A7C333C5F066
:2024820033C5F079007A001200EA89828A83E0A3F5F0E0C5F078FD1200B6F608A6F018E67F
:2024A2000886F0901888F078F51200B6E60886F0C0E0C0F01239C6158115817FFA0200D10A
:2024C2007F091200C2E4F5F078F81200B6F608A6F0123FA2122F90901872E0A3F5F0E0C51E
:2024E200F09018741200DC1201E47003022508901872E0A3F5F0E0C5F0901874F0A3C5F0CC
:20250200F0C5F0122F90E4F5F0798C7A181200EAC001C002125A01D083D082F07B007C006B
:202522001201E47003022F4FE4F5F0798C7A181200EA89828A83E01200FAC0E0C0F0125A93
:202542001515811581902F230201031203E3901888E075F000C0E0C0F0121E6415811581D3
:20256200E4F5F078F61200B6F608A6F0E4F5F008F608A6F0901876E054FB901876F054F7BB
:20258200901876F0547F901876F04402901876F0E475F0C0C0E0C0F0901876E075F000C07A
:2025A200E0C0F012599A15811581158115811203E390187FE075F000C0E0C0F0741575F08A
:2025C20000C0E0C0F0901880E075F000C0E0C0F01207237FFA1200C2120268901882E0A33A
:2025E200F5F0E0C5F078FA1200B6F608A6F078F61200B6E60886F045F0600302265E125A6D
:202602000145F0700302263078F81200B6E60886F012019918F608A6F01201A7181818E6DB
:202622000886F012019918F608A6F01201A7E5088509F078FA1200B686030886041201FB3A
:20264200700302265B78F61200B6E60886F012019918F608A6F01201A70225F078F812003D
:20266200B6E60886F045F0600302283290186FE054041200FA1201BA45F0600C901870E089
:2026820054801200FA1201BA45F060030226EC740275F000C0E0C0F012028D158115819057
:2026A200186FE054041200FA1201BA45F0600C901870E054801200FA1201BA45F0600302A0
:2026C20026EC901876E04480901876F0E475F0C0C0E0C0F0901876E075F000C0E0C0F012F8
:2026E200599A1581158115811581901881E075F000C0E0C0F0741475F000C0E0C0F0E4C0EE
:20270200E0C0F01207237FFA1200C2C294D293901876E054FD901876F04408901876F054D8
:20272200FB901876F0E475F0C0C0E0C0F0901876E075F000C0E0C0F012599A15811581153C
:20274200811581E4F5F078F61200B6F608A6F012026878F61200B6E60886F045F06003021D
:202762002832125A0145F0700302278278F61200B6E60886F012019918F608A6F01201A791
:20278200901872E0A3F5F0E0C5F09018741200DC1201E470030227B1901872E0A3F5F0E070
:2027A200C5F0901874F0A3C5F0F0C5F0122F9090186FE054041200FA1201BA45F0600C902F
:2027C2001870E054801200FA1201BA45F0600302282F740275F000C0E0C0F012028D15818F
:2027E200158190186FE054041200FA1201BA45F0600C901870E054801200FA1201BA45F09E
:20280200600302282F901876E04480901876F0E475F0C0C0E0C0F0901876E075F000C0E0CE
:20282200C0F012599A158115811581158102275478F81200B6E60886F045F0600302294568
:20284200E4F5F0181818F608A6F0C293D294901884E078FE1200B6F6901885E0A3F5F0E061
:20286200C5F01818F608A6F01203E3901887E075F000C0E0C0F0121E641581158178FE12D9
:2028820000B6E675F000C0E0C0F07414C0E0C0F012062D1581158115811581120268125A88
:2028A2000145F070030228D078F81200B6E60886F012019918F608A6F01201A7181818E697
:2028C2000886F012019918F608A6F01201A7E5088509F078FC1200B686030886041201FB96
:2028E20070030228F5740175F00078F61200B6F608A6F078F61200B6E60886F045F070035E
:202902000228A0D295D293D293901876E054FD901876F054F7901876F054FB901876F05453
:202922007F901876F0E475F0C0C0E0C0F0901876E075F000C0E0C0F012599A1581158115B6
:2029420081158178F81200B6E60886F045F060030229D8E4F5F0181818F608A6F0D293D24B
:202962009490187CE078FE1200B6F690187DE0A3F5F0E0C5F01818F608A6F008E675F00050
:20298200C0E0C0F07414C0E0C0F01205371581158115811581120268E5088509F078FC12FA
:2029A20000B686030886041201FB70030229C578F61200B6E60886F012019918F608A6F0E1
:2029C2001201A778F61200B6E60886F045F0700302299A1203E31203E3D293D2949018765B
:2029E200E054FD901876F054F7901876F054FB901876F0547F901876F0E475F0C0C0E0C096
:202A0200F0901876E075F000C0E0C0F012599A1581158115811581E4F5F078F81200B6F6BD
:202A220008A6F0022F4F1203E3901887E075F000C0E0C0F0121E6415811581E4F5F078F6C3
:202A42001200B6F608A6F0901876E054FB901876F054F7901876F0547F901876F0440290AD
:202A62001876F0E475F0C0C0E0C0F0901876E075F000C0E0C0F012599A15811581158115EE
:202A820081901877E075F000C0E0C0F0741575F000C0E0C0F012062D158115811581158124
:202AA20012026890187AE0A3F5F0E0C5F078FA1200B6F608A6F078F61200B6E60886F045CC
:202AC200F06003022B26125A0145F07003022AF878F81200B6E60886F012019918F608A611
:202AE200F01201A7181818E60886F012019918F608A6F01201A7E5088509F078FA1200B6C7
:202B020086030886041201FB7003022B2378F61200B6E60886F012019918F608A6F01201C2
:202B2200A7022AB878F81200B6E60886F045F06003022CF890186FE054041200FA1201BA86
:202B420045F0600C901870E054801200FA1201BA45F06003022BB4740275F000C0E0C0F089
:202B620012028D1581158190186FE054041200FA1201BA45F0600C901870E054801200FAE5
:202B82001201BA45F06003022BB4901876E04480901876F0E475F0C0C0E0C0F0901876E0C6
:202BA20075F000C0E0C0F012599A1581158115811581901879E075F000C0E0C0F07414754E
:202BC200F000C0E0C0F012062D1581158115811581C293D294901876E054FD901876F054AA
:202BE200F7901876F04404901876F0E475F0C0C0E0C0F0901876E075F000C0E0C0F0125901
:202C02009A1581158115811581E4F5F078F61200B6F608A6F012026878F61200B6E6088607
:202C2200F045F06003022CF8125A0145F07003022C4878F61200B6E60886F012019918F605
:202C420008A6F01201A7901872E0A3F5F0E0C5F09018741200DC1201E47003022C77901842
:202C620072E0A3F5F0E0C5F0901874F0A3C5F0F0C5F0122F9090186FE054041200FA12019B
:202C8200BA45F0600C901870E054801200FA1201BA45F06003022CF5740275F000C0E0C03C
:202CA200F012028D1581158190186FE054041200FA1201BA45F0600C901870E054801200AE
:202CC200FA1201BA45F06003022CF5901876E04480901876F0E475F0C0C0E0C0F090187629
:202CE200E075F000C0E0C0F012599A1581158115811581022C1A78F81200B6E60886F045B7
:202D0200F06003022D8BE4F5F0181818F608A6F0D293D29490187CE078FE1200B6F6901854
:202D22007DE0A3F5F0E0C5F01818F608A6F008E675F000C0E0C0F07414C0E0C0F01205378A
:202D42001581158115811581120268E5088509F078FC1200B686030886041201FB70030258
:202D62002D7878F61200B6E60886F012019918F608A6F01201A778F61200B6E60886F04521
:202D8200F07003022D4D1203E3D293D294901876E054FD901876F054F7901876F054FB90FA
:202DA2001876F0547F901876F0E475F0C0C0E0C0F0901876E075F000C0E0C0F012599A158C
:202DC200811581158115811203E3E4F5F078F81200B6F608A6F0022F4FE4C0E0C0E0121E4D
:202DE2006415811581022F4F740175F000C0E0C0F0121EE6158115811203E3743C75F00048
:202E0200C0E0C0F0121E6415811581124163740175F000C0E0C0F01239C615811581022F52
:202E22004F740275F000C0E0C0F0121EE6158115811203E3743C75F000C0E0C0F0121E64E3
:202E420015811581124163740275F000C0E0C0F01239C615811581022F4F740375F000C00A
:202E6200E0C0F0121EE6158115811203E3743C75F000C0E0C0F0121E6415811581124163AB
:202E8200740375F000C0E0C0F01239C615811581022F4F1241631203E3901887E075F00025
:202EA200C0E0C0F0121E6415811581123FA2022F4F1248ED022F4F741B75F000C0E0C0F082
:202EC2001259BA15811581744975F008C0E0C0F01259DA15811581741B75F000C0E0C0F070
:202EE2001259BA15811581745075F008C0E0C0F01259DA15811581745375F008C0E0C0F009
:202F02001259DA15811581022F4F78F81200B6E60886F012019918F608A6F01201A7022FDF
:202F22004F0C2F5800B92E4900B32E5200952E50005C2E3300232E3200EA2D3100DB2D3077
:202F420000282A42004D25410000004F2F90186EE0540175F00045F0700690186EE0540203
:202F62007003022F7B78F81200B6E60886F012019918F608A6F01201A778F81200B6E6085C
:202F820086F045F070030224D97FF70200D1058112586278FE1200B6F6741B75F000C0E0AF
:202FA200C0F01259BA15811581748C75F008C0E0C0F01259DA15811581749275F008C0E0CD
:202FC200C0F078FC1200B6E675F000C0E0C0F0740212584E1581158115811581741B75F0EE
:202FE20000C0E0C0F01259BA15811581749675F008C0E0C0F01259DA15811581749E75F07F
:2030020008C0E0C0F078FC1200B6E6540175F000C0E0C0F0740275F00012584E158115816B
:2030220015811581741B75F000C0E0C0F01259BA1581158174A275F008C0E0C0F01259DAB5
:203042001581158174AA75F008C0E0C0F078FC1200B6E6540275F0007B017C00120187C038
:20306200E0C0F0740275F00012584E1581158115811581741B75F000C0E0C0F01259BA1555
:2030820081158174AE75F008C0E0C0F01259DA1581158174B675F008C0E0C0F078FC12005A
:2030A200B6E6540475F0007B027C00120187C0E0C0F0740275F00012584E1581158115817D
:2030C2001581741B75F000C0E0C0F01259BA1581158174BA75F008C0E0C0F01259DA1581FD
:2030E200158174C275F008C0E0C0F078FC1200B6E6540875F0007B037C00120187C0E0C06E
:20310200F0740275F00012584E1581158115811581741B75F000C0E0C0F01259BA158115BE
:203122008174C675F008C0E0C0F01259DA1581158174CE75F008C0E0C0F078FC1200B6E683
:20314200541075F0007B047C00120187C0E0C0F0740275F00012584E1581158115811581D4
:2031620012586878FE1200B6F6741B75F000C0E0C0F01259BA1581158174D275F008C0E05F
:20318200C0F01259DA1581158174D975F008C0E0C0F078FC1200B6E675F000C0E0C0F074B7
:2031A2000212584E1581158115811581741B75F000C0E0C0F01259BA1581158174DD75F0B0
:2031C20008C0E0C0F01259DA1581158174E575F008C0E0C0F078FC1200B6E6541075F00023
:2031E2007B047C00120187C0E0C0F0740275F00012584E158115811581158112586B78FEB2
:203202001200B6F6741B75F000C0E0C0F01259BA1581158174E975F008C0E0C0F01259DAFA
:203222001581158174F075F008C0E0C0F078FC1200B6E675F000C0E0C0F0740212584E1525
:2032420081158115811581741B75F000C0E0C0F01259BA1581158174F475F008C0E0C0F06F
:203262001259DA1581158174FB75F008C0E0C0F078FC1200B6E6540175F000C0E0C0F0740F
:203282000275F00012584E1581158115811581741B75F000C0E0C0F01259BA1581158174AC
:2032A200FF75F008C0E0C0F01259DA15811581740675F009C0E0C0F078FC1200B6E654022F
:2032C20075F0007B017C00120187C0E0C0F0740275F00012584E1581158115811581741B2B
:2032E20075F000C0E0C0F01259BA15811581740A75F009C0E0C0F01259DA15811581741194
:2033020075F009C0E0C0F078FC1200B6E6540475F0007B027C00120187C0E0C0F074027540
:20332200F00012584E1581158115811581741B75F000C0E0C0F01259BA15811581741575F8
:20334200F009C0E0C0F01259DA15811581741C75F009C0E0C0F078FC1200B6E6540875F080
:20336200007B037C00120187C0E0C0F0740275F00012584E1581158115811581741B75F088
:2033820000C0E0C0F01259BA15811581742075F009C0E0C0F01259DA15811581742775F0C7
:2033A20009C0E0C0F078FC1200B6E6541075F0007B047C00120187C0E0C0F0740275F00007
:2033C20012584E1581158115811581741B75F000C0E0C0F01259BA15811581742B75F00939
:2033E200C0E0C0F01259DA15811581743375F009C0E0C0F078FC1200B6E6542075F0007B2F
:20340200057C00120187C0E0C0F0740275F00012584E1581158115811581741B75F000C0A0
:20342200E0C0F01259BA15811581743775F009C0E0C0F01259DA15811581743F75F009C0EE
:20344200E0C0F078FC1200B6E6544075F0007B067C00120187C0E0C0F0740275F000125893
:203462004E1581158115811581741B75F000C0E0C0F01259BA15811581744375F009C0E04A
:20348200C0F01259DA15811581744B75F009C0E0C0F078FC1200B6E6548075F0007B077C33
:2034A20000120187C0E0C0F0740275F00012584E158115811581158112586E78FE1200B61F
:2034C200F6741B75F000C0E0C0F01259BA15811581744F75F009C0E0C0F01259DA158115EE
:2034E20081745675F009C0E0C0F078FC1200B6E675F000C0E0C0F0740212584E1581158190
:2035020015811581741B75F000C0E0C0F01259BA15811581745A75F009C0E0C0F01259DA17
:2035220015811581746275F009C0E0C0F078FC1200B6E6540175F000C0E0C0F0740275F0C2
:203542000012584E1581158115811581741B75F000C0E0C0F01259BA15811581746675F085
:2035620009C0E0C0F01259DA15811581746E75F009C0E0C0F078FC1200B6E6540275F00002
:203582007B017C00120187C0E0C0F0740275F00012584E1581158115811581741B75F00068
:2035A200C0E0C0F01259BA15811581747275F009C0E0C0F01259DA15811581747A75F009F7
:2035C200C0E0C0F078FC1200B6E6540475F0007B027C00120187C0E0C0F0740275F00012EA
:2035E200584E1581158115811581741B75F000C0E0C0F01259BA15811581747E75F009C016
:20360200E0C0F01259DA15811581748675F009C0E0C0F078FC1200B6E6540875F0007B038E
:203622007C00120187C0E0C0F0740275F00012584E1581158115811581741B75F000C0E0A3
:20364200C0F01259BA15811581748A75F009C0E0C0F01259DA15811581749275F009C0E026
:20366200C0F078FC1200B6E6541075F0007B047C00120187C0E0C0F0740275F00012584E35
:203682001581158115811581741B75F000C0E0C0F01259BA15811581749675F009C0E0C063
:2036A200F01259DA15811581749E75F009C0E0C0F078FC1200B6E6542075F0007B057C00E0
:2036C200120187C0E0C0F0740275F00012584E1581158115811581741B75F000C0E0C0F0CF
:2036E2001259BA1581158174A275F009C0E0C0F01259DA1581158174AA75F009C0E0C0F056
:2037020078FC1200B6E6544075F0007B067C00120187C0E0C0F0740275F00012584E15817C
:20372200158115811581741B75F000C0E0C0F01259BA1581158174AE75F009C0E0C0F0123E
:2037420059DA1581158174B675F009C0E0C0F078FC1200B6E6548075F0007B077C001201B4
:2037620087C0E0C0F0740275F00012584E1581158115811581741B75F000C0E0C0F01259D6
:20378200BA1581158174BA75F009C0E0C0F01259DA1581158174C075F009C0E0C0F0E47599
:2037A200F0C0C0E0C0F0125979158115815440C5F05400C5F07B067C00120187C0E0C0F0BE
:2037C200740275F00012584E1581158115811581741B75F000C0E0C0F01259BA1581158167
:2037E20074C475F009C0E0C0F01259DA1581158174CB75F009C0E0C0F0E475F0C0C0E0C0FA
:20380200F012597915811581543FC5F05400C0F0C0E0740275F00012584E15811581158165
:203822001581741B75F000C0E0C0F01259BA1581158174CF75F009C0E0C0F01259DA15817F
:20384200158174D675F009C0E0C0F0E475F0D0C0E0C0F0125979158115815440C5F05400B2
:20386200C5F07B067C00120187C0E0C0F0740275F00012584E1581158115811581741B75BB
:20388200F000C0E0C0F01259BA1581158174DA75F009C0E0C0F01259DA1581158174E1754E
:2038A200F009C0E0C0F0E475F0D0C0E0C0F012597915811581543FC5F05400C0F0C0E074E4
:2038C2000275F00012584E1581158115811581741B75F000C0E0C0F01259BA158115817466
:2038E200E575F009C0E0C0F01259DA1581158174EC75F009C0E0C0F0E475F0E0C0E0C0F01B
:20390200125979158115815440C5F05400C5F07B067C00120187C0E0C0F0740275F000126F
:20392200584E1581158115811581741B75F000C0E0C0F01259BA1581158174F075F009C060
:20394200E0C0F01259DA1581158174F775F009C0E0C0F0E475F0E0C0E0C0F0125979158148
:203962001581543FC5F05400C0F0C0E0740275F00012584E1581158115811581741B75F0E4
:2039820000C0E0C0F01259BA1581158174FB75F009C0E0C0F01259DA15811581740275F00B
:2039A2000AC0E0C0F0901872E0A3F5F0E0C0F0C0E0740275F00012584E158115811581158F
:2039C20081158122741B75F000C0E0C0F01259BA15811581740675F00AC0E0C0F01259DA99
:2039E20015811581740E75F00AC0E0C0F01259DA15811581741B75F000C0E0C0F01259BA7E
:203A020015811581741075F00AC0E0C0F01259DA15811581741875F00AC0E0C0F01259DA34
:203A220015811581741B75F000C0E0C0F01259BA15811581741A75F00AC0E0C0F01259DA31
:203A420015811581742275F00AC0E0C0F01259DA1581158178FB1200B6E60886F07B017CDB
:203A6200001201DC7003023A9B741B75F000C0E0C0F01259BA15811581742475F00AC0E0CF
:203A8200C0F01259DA15811581742C75F00AC0E0C0F01259DA1581158178FB1200B6E6080A
:203AA20086F07B027C001201DC7003023AE0741B75F000C0E0C0F01259BA15811581742EE0
:203AC20075F00AC0E0C0F01259DA15811581743675F00AC0E0C0F01259DA1581158178FB67
:203AE2001200B6E60886F07B037C001201DC7003023B25741B75F000C0E0C0F01259BA155C
:203B0200811581743875F00AC0E0C0F01259DA15811581744075F00AC0E0C0F01259DA15E3
:203B2200811581741B75F000C0E0C0F01259BA15811581744275F00AC0E0C0F01259DA1508
:203B4200811581744A75F00AC0E0C0F0901877E075F000C0E0C0F0740275F00012584E1573
:203B620081158115811581741B75F000C0E0C0F01259BA15811581744E75F00AC0E0C0F0EA
:203B82001259DA15811581745675F00AC0E0C0F0901878E075F000C0E0C0F0740275F00099
:203BA20012584E1581158115811581741B75F000C0E0C0F01259BA15811581745A75F00A21
:203BC200C0E0C0F01259DA15811581746275F00AC0E0C0F0901879E075F000C0E0C0F07463
:203BE2000275F00012584E1581158115811581741B75F000C0E0C0F01259BA158115817443
:203C02006675F00AC0E0C0F01259DA15811581746E75F00AC0E0C0F090187AE0A3F5F0E001
:203C2200C0F0C0E0740275F00012584E1581158115811581741B75F000C0E0C0F01259BADE
:203C420015811581747275F00AC0E0C0F01259DA15811581747A75F00AC0E0C0F090187C4F
:203C6200E075F000C0E0C0F0740275F00012584E1581158115811581741B75F000C0E0C06E
:203C8200F01259BA15811581747E75F00AC0E0C0F01259DA15811581748675F00AC0E0C0F6
:203CA200F090187DE0A3F5F0E0C0F0C0E0740275F00012584E1581158115811581741B7566
:203CC200F000C0E0C0F01259BA15811581748A75F00AC0E0C0F01259DA15811581901887F4
:203CE200E075F000903D5E020103749275F00AC0E0C0F01259DA15811581023D7A749775DD
:203D0200F00AC0E0C0F01259DA15811581023D7A749C75F00AC0E0C0F01259DA15811581ED
:203D2200023D7A74A175F00AC0E0C0F01259DA15811581023D7A74A675F00AC0E0C0F012DF
:203D420059DA15811581023D7A74AB75F00AC0E0C0F01259DA15811581023D7A4B3D1200A7
:203D6200383D0300253D0100123D0000FF3C0F00EC3C020000007A3D741B75F000C0E0C098
:203D8200F01259BA1581158174B075F00AC0E0C0F01259DA1581158174B875F00AC0E0C091
:203DA200F090187FE075F000C0E0C0F0740275F00012584E1581158115811581741B75F076
:203DC20000C0E0C0F01259BA1581158174BC75F00AC0E0C0F01259DA1581158174C475F043
:203DE2000AC0E0C0F0901880E075F000C0E0C0F0740275F00012584E1581158115811581BF
:203E0200741B75F000C0E0C0F01259BA1581158174C875F00AC0E0C0F01259DA158115819F
:203E220074D075F00AC0E0C0F0901881E075F000C0E0C0F0740275F00012584E1581158100
:203E420015811581741B75F000C0E0C0F01259BA1581158174D475F00AC0E0C0F01259DA53
:203E62001581158174DC75F00AC0E0C0F0901882E0A3F5F0E0C0F0C0E0740275F0001258FE
:203E82004E1581158115811581741B75F000C0E0C0F01259BA1581158174E075F00AC0E082
:203EA200C0F01259DA1581158174E875F00AC0E0C0F0901884E075F000C0E0C0F074027518
:203EC200F00012584E1581158115811581741B75F000C0E0C0F01259BA1581158174EC7576
:203EE200F00AC0E0C0F01259DA1581158174F475F00AC0E0C0F0901885E0A3F5F0E0C0F0B9
:203F0200C0E0740275F00012584E1581158115811581741B75F000C0E0C0F01259BA158115
:203F2200158174F875F00AC0E0C0F01259DA15811581901888E075F000903F8D0201037402
:203F42000075F00BC0E0C0F01259DA15811581023FA1740575F00BC0E0C0F01259DA158138
:203F62001581023FA1740A75F00BC0E0C0F01259DA15811581023FA1740F75F00BC0E0C0E3
:203F8200F01259DA15811581023FA17A3F1D00673F0D00543F0C00413F05000000A13F222D
:203FA200741B75F000C0E0C0F01259BA15811581741475F00BC0E0C0F01259DA15811581B1
:203FC200741B75F000C0E0C0F01259BA15811581741875F00BC0E0C0F01259DA158115818D
:203FE200741B75F00BC0E0C0F01259DA15811581746B75F00BC0E0C0F01259DA15811581EF
:2040020074BC75F00BC0E0C0F01259DA15811581740D75F00CC0E0C0F01259DA158115818A
:20402200745E75F00CC0E0C0F01259DA1581158174AF75F00CC0E0C0F01259DA1581158125
:20404200740075F00DC0E0C0F01259DA15811581745175F00DC0E0C0F01259DA15811581BF
:2040620074A275F00DC0E0C0F01259DA1581158174F375F00DC0E0C0F01259DA158115815B
:20408200744475F00EC0E0C0F01259DA15811581749575F00EC0E0C0F01259DA15811581F5
:2040A20074E675F00EC0E0C0F01259DA15811581743775F00FC0E0C0F01259DA1581158190
:2040C200748875F00FC0E0C0F01259DA1581158174D975F00FC0E0C0F01259DA158115812B
:2040E200742A75F010C0E0C0F01259DA15811581747B75F010C0E0C0F01259DA15811581C5
:2041020074CC75F010C0E0C0F01259DA15811581741D75F011C0E0C0F01259DA158115815F
:20412200746E75F011C0E0C0F01259DA1581158174BF75F011C0E0C0F01259DA15811581FA
:20414200741075F012C0E0C0F01259DA15811581746175F012C0E0C0F01259DA1581158194
:204162002205810581E4F5F078FD1200B6F608A6F0124641748C75F018C0E0C0F074017525
:20418200F000C0E0C0F0125A471581158115811581E4F5F0798C7A181200EA89828A83E07E
:2041A2001200FAC0E0C0F0125A15158115819045C1020103746A75F012C0E0C0F0740175C9
:2041C200F00012584E15811581748C75F018C0E0C0F0740475F000C0E0C0F0125A471581C6
:2041E200158115811581748C75F018C0E0C0F0125AA815811581901877F01246410245FD02
:20420200748C75F012C0E0C0F0740175F00012584E15811581748C75F018C0E0C0F07404D2
:2042220075F000C0E0C0F0125A471581158115811581748C75F018C0E0C0F0125AA8158145
:204242001581901879F01246410245FD74B475F012C0E0C0F0740175F00012584E158115AC
:2042620081748C75F018C0E0C0F0740475F000C0E0C0F0125A471581158115811581748CB6
:2042820075F018C0E0C0F0125AA81581158190187AF0A3C5F0F0C5F01246410245FD74D4DB
:2042A20075F012C0E0C0F0740175F00012584E15811581748C75F018C0E0C0F0740475F0CD
:2042C20000C0E0C0F0125A471581158115811581748C75F018C0E0C0F0125AA81581158174
:2042E20090187CF01246410245FD74F975F012C0E0C0F0740175F00012584E158115817465
:204302008C75F018C0E0C0F0740475F000C0E0C0F0125A471581158115811581748C75F0A5
:2043220018C0E0C0F0125AA81581158190187DF0A3C5F0F0C5F01246410245FD741B75F0F0
:2043420013C0E0C0F0740175F00012584E15811581748C75F018C0E0C0F0740475F000C0D0
:20436200E0C0F0125A471581158115811581748C75F018C0E0C0F0125AA8158115819018EB
:204382007FF01246410245FD743C75F013C0E0C0F0740175F00012584E15811581748C7524
:2043A200F018C0E0C0F0740475F000C0E0C0F0125A471581158115811581748C75F018C02E
:2043C200E0C0F0125AA815811581901880F01246410245FD746675F013C0E0C0F07401758A
:2043E200F00012584E15811581748C75F018C0E0C0F0740475F000C0E0C0F0125A471581A4
:20440200158115811581748C75F018C0E0C0F0125AA815811581901881F01246410245FDD5
:20442200748D75F013C0E0C0F0740175F00012584E15811581748C75F018C0E0C0F07404AE
:2044420075F000C0E0C0F0125A471581158115811581748C75F018C0E0C0F0125AA8158123
:204462001581901882F0A3C5F0F0C5F01246410245FD74AF75F013C0E0C0F0740175F000EB
:2044820012584E15811581748C75F018C0E0C0F0740475F000C0E0C0F0125A47158115815D
:2044A20015811581748C75F018C0E0C0F0125AA815811581901884F01246410245FD74CE86
:2044C20075F013C0E0C0F0740175F00012584E15811581748C75F018C0E0C0F0740475F0AA
:2044E20000C0E0C0F0125A471581158115811581748C75F018C0E0C0F0125AA81581158152
:20450200901885F0A3C5F0F0C5F01246410245FD74EB75F013C0E0C0F0740175F000125837
:204522004E15811581748C75F018C0E0C0F0740575F000C0E0C0F0125A471581158115818F
:204542001581748C75F018C0E0C0F0125AA815811581901887F01246410245FD740E75F0D3
:2045620014C0E0C0F0740175F00012584E15811581748C75F018C0E0C0F0740575F000C0AC
:20458200E0C0F0125A471581158115811581748C75F018C0E0C0F0125AA8158115819018C9
:2045A20088F01246410245FD78FD1200B6E60886F012019918F608A6F01201A70245FDAA03
:2045C2004558005E454F0012454E00C0444D0074444C0022444900D64348008A4347003EEE
:2045E200434600EC424500A04244004E42430002424200B64141000000FD4590186EE0547A
:204602000175F00045F0700690186EE05402700302462978FD1200B6E60886F012019918F2
:20462200F608A6F01201A778FD1200B6E60886F045F07003024176123FA215811581227473
:204642001B75F000C0E0C0F01259BA15811581743275F014C0E0C0F01259DA1581158174E3
:204662001B75F000C0E0C0F01259BA15811581743675F014C0E0C0F01259DA1581158174BF
:204682003975F014C0E0C0F0740175F00012584E15811581748A75F014C0E0C0F0740175A7
:2046A200F00012584E1581158174DB75F014C0E0C0F0740175F00012584E15811581742CAE
:2046C20075F015C0E0C0F0740175F00012584E15811581747D75F015C0E0C0F0740175F0BB
:2046E2000012584E1581158174CE75F015C0E0C0F0740175F00012584E1581158174D07551
:20470200F015C0E0C0F0901877E075F000C0E0C0F0740275F00012584E1581158115811524
:2047220081740275F016C0E0C0F0901879E075F000C0E0C0F0740275F00012584E158115C1
:204742008115811581743475F016C0E0C0F090187AE0A3F5F0E0C0F0C0E0740275F0001290
:20476200584E1581158115811581746675F016C0E0C0F090187CE075F000C0E0C0F0740265
:2047820075F00012584E1581158115811581749875F016C0E0C0F090187DE0A3F5F0E0C09E
:2047A200F0C0E0740275F00012584E158115811581158174CA75F016C0E0C0F090187FE06C
:2047C20075F000C0E0C0F0740275F00012584E158115811581158174FC75F016C0E0C0F0FC
:2047E200901880E075F000C0E0C0F0740275F00012584E1581158115811581742E75F017F1
:20480200C0E0C0F0901881E075F000C0E0C0F0740275F00012584E15811581158115817429
:204822006075F017C0E0C0F0901882E0A3F5F0E0C0F0C0E0740275F00012584E15811581C9
:2048420015811581749275F017C0E0C0F0901884E075F000C0E0C0F0740275F00012584E04
:20486200158115811581158174C475F017C0E0C0F0901885E0A3F5F0E0C0F0C0E07402752A
:20488200F00012584E158115811581158174F675F017C0E0C0F0901887E075F000C0E0C00C
:2048A200F0740275F00012584E1581158115811581742975F018C0E0C0F0901888E075F03C
:2048C20000C0E0C0F0740275F00012584E1581158115811581745C75F018C0E0C0F0740189
:2048E20075F00012584E15811581220581125A0145F060030249E9122F90E478FE1200B699
:20490200F678FE1200B6E675F0007B057C001201ED700C02494378FE1200B6E60680E27410
:204922000175F00078FE1200B686037C00120179C0E0C0F0121E6415811581122F90024914
:2049420018D2C5D2C6122F90E478FE1200B6F678FE1200B6E675F0007B057C001201ED7030
:204962000C02499178FE1200B6E60680E2740175F00078FE1200B686037C00120179C0E078
:20498200C0F0121E6415811581122F90024966C2C5D2C6122F90E478FE1200B6F678FE1293
:2049A20000B6E675F0007B057C001201ED700C0249DF78FE1200B6E60680E2740175F000EC
:2049C20078FE1200B686037C00120179C0E0C0F0121E6415811581122F900249B4C2C5C2DD
:2049E200C6122F900248EF15812243871075FF01B2971254621203E3125A017B207C00123F
:204A020001DC7003024A1F1203E3740175F000C0E0C0F0121EE6158115811224C290187164
:204A2200E054017003024BC71203E3740175F000C0E0C0F0121EE615811581740275F00079
:204A4200C0E0C0F012028D15811581901871E054017003024BC7125A017B207C001201DCEF
:204A62007003024A7D1203E31224C2740175F000C0E0C0F01239C61581158190186EE05457
:204A82000175F00045F06006901871E054087003024AC8740275F000C0E0C0F012028D1556
:204AA20081158190186EE0540175F00045F06006901871E054087003024AC87401F50D74CB
:204AC20001F50E124F1E90186EE0540175F00045F0600C901871E054081200FA1201BA458D
:204AE200F07003024B22740275F000C0E0C0F012028D1581158190186EE0540175F00045F5
:204B0200F0600C901871E054081200FA1201BA45F07003024B227401F50DE4F50E124F1E15
:204B220090186EE0540275F00045F06006901871E054087003024B6B740275F000C0E0C06C
:204B4200F012028D1581158190186EE0540275F00045F06006901871E054087003024B6BCA
:204B6200E4F50DE4F50E124F1E90186EE0540275F00045F0600C901871E054081200FA1222
:204B820001BA45F07003024BC4740275F000C0E0C0F012028D1581158190186EE0540275E6
:204BA200F00045F0600C901871E054081200FA1201BA45F07003024BC4E4F50DE4F50E129C
:204BC2004F1E024A4D901871E054027003024D721203E3740275F000C0E0C0F0121EE615FC
:204BE2008115811203E3740275F000C0E0C0F012028D15811581901871E054027003024D9B
:204C020072125A017B207C001201DC7003024C281203E31224C2740275F000C0E0C0F01297
:204C220039C61581158190186EE0540175F00045F06006901871E054087003024C737402FD
:204C420075F000C0E0C0F012028D1581158190186EE0540175F00045F06006901871E05438
:204C6200087003024C737401F50D7401F50E124F1E90186EE0540175F00045F0600C90188F
:204C820071E054081200FA1201BA45F07003024CCD740275F000C0E0C0F012028D15811552
:204CA2008190186EE0540175F00045F0600C901871E054081200FA1201BA45F07003024CFC
:204CC200CD7401F50DE4F50E124F1E90186EE0540275F00045F06006901871E05408700314
:204CE200024D16740275F000C0E0C0F012028D1581158190186EE0540275F00045F0600609
:204D0200901871E054087003024D16E4F50DE4F50E124F1E90186EE0540275F00045F060D2
:204D22000C901871E054081200FA1201BA45F07003024D6F740275F000C0E0C0F012028D05
:204D42001581158190186EE0540275F00045F0600C901871E054081200FA1201BA45F07000
:204D620003024D6FE4F50DE4F50E124F1E024BF8901871E054047003024F1A1203E3740341
:204D820075F000C0E0C0F0121EE615811581740275F000C0E0C0F012028D1581158190187A
:204DA20071E054047003024F1A125A017B207C001201DC7003024DD01203E31224C27403FE
:204DC20075F000C0E0C0F01239C61581158190186EE0540175F00045F06006901871E05447
:204DE200087003024E1B740275F000C0E0C0F012028D1581158190186EE0540175F00045DE
:204E0200F06006901871E054087003024E1B7401F50D7401F50E124F1E90186EE0540175D9
:204E2200F00045F0600C901871E054081200FA1201BA45F07003024E75740275F000C0E0C9
:204E4200C0F012028D1581158190186EE0540175F00045F0600C901871E054081200FA120F
:204E620001BA45F07003024E757401F50DE4F50E124F1E90186EE0540275F00045F06006DF
:204E8200901871E054087003024EBE740275F000C0E0C0F012028D1581158190186EE054F8
:204EA2000275F00045F06006901871E054087003024EBEE4F50DE4F50E124F1E90186EE0D6
:204EC200540275F00045F0600C901871E054081200FA1201BA45F07003024F17740275F05B
:204EE20000C0E0C0F012028D1581158190186EE0540275F00045F0600C901871E0540812DA
:204F020000FA1201BA45F07003024F17E4F50DE4F50E124F1E024DA00249FA227F0612007F
:204F2200C2E4F5F078F91200B6F608A6F0E4F5F0080808F608A6F0E50E7003024FA612082B
:204F42005A78FB1200B6F608A6F018E60886F0904F92020103024FA6024FA6E4C0E0C0E021
:204F62001216971581158190186EE054027003024F7DE4F50E120ED1024FA6E4C0E0C0E0C4
:204F8200121A691581158102545D121D6E02545D8C4FF3FF5D4FF1FF5A4FF0FF574F0100A3
:204FA2000000A64FE50E600302504490186EE054026003024FFA120C3778FB1200B6F60886
:204FC200A6F018E60886F0904FE7020103024FF7E4C0E0C0E0121A691581158102545D12FF
:204FE2001D6E02545DE14FF3FFD24FF2FFCF4F01000000F74F025044120F9878FB1200B64E
:20500200F608A6F018E60886F090503402010302504490186EE05402600302502BE4C0E01E
:20502200C0E0121A691581158102545D121D6E02545D2E50F3FF1450F2FF115001000000E3
:205042004450120268740175F00045F0700302545A901872E0A3F5F0E0C5F078FD1200B6B8
:2050620086030886041201E47003025181901872E0A3F5F0E0C5F018F608A6F0901870E01A
:2050820054801200FA1201BA45F06003025181901876E04402901876F0E50E60030250C437
:2050A200901877E075F000C0E0C0F0741475F000C0E0C0F012062D1581158115811581025E
:2050C20050EB90187FE075F000C0E0C0F0741475F000C0E0C0F0901880E075F000C0E0C0CD
:2050E200F01207237FFA1200C2742C75F001C0E0C0F012028D15811581901876E054FD9033
:205102001876F0901870E054801200FA1201BA45F06003025131E50E700302512BE4C0E0E6
:20512200C0E012169715811581121C7502545DE50E600302515A901879E075F000C0E0C0C3
:20514200F0741475F000C0E0C0F012062D1581158115811581025181901881E075F000C081
:20516200E0C0F0741475F000C0E0C0F0901880E075F000C0E0C0F01207237FFA1200C2E535
:205182000E60030252F690186EE0540175F00045F0700690186EE05402600302523074024E
:2051A20075F000C0E0C0F012028D1581158190186EE0540175F00045F0700690186EE054C6
:2051C20002600302523074D075F007C0E0C0F0121A691581158178FB1200B6F608A6F0183C
:2051E200E60886F0905218020103120F4602545DE50D75F0007B007C001201DC6003025439
:205202005D120ED1025230120ED1025230025230120F4602545D1252EFFF0F52F6FF0952A4
:20522200F4FFF251F5FFEC5101000000305290186EE0540175F00045F06006901871E054EA
:205242000870030252B2740275F000C0E0C0F012028D1581158190186EE0540175F00045DE
:20526200F06006901871E0540870030252B212139878FB1200B6F608A6F07401F50E18E606
:205282000886F07B017C001201DC7003025297120BDD0252B2E4C0E0C0E0121697158115BB
:2052A2008178FB1200B6F608A6F0E4F50E120ED190186EE0540275F00045F060069018715F
:2052C200E0540870030252F6740275F000C0E0C0F012028D1581158190186EE0540275F02A
:2052E2000045F06006901871E0540870030252F6C294D293E50E700302545790186EE054E7
:205302000175F00045F0700690186EE054026003025356740275F000C0E0C0F012028D153F
:2053220081158190186EE0540175F00045F0700690186EE05402600302535674D075F007EF
:20534200C0E0C0F01216971581158178FB1200B6F608A6F090186EE0540175F00045F060FC
:205362000C901871E054081200FA1201BA45F070030253BF740275F000C0E0C0F012028D69
:205382001581158190186EE0540175F00045F0600C901871E054081200FA1201BA45F070BB
:2053A200030253BF74D075F007C0E0C0F01216971581158178FB1200B6F608A6F090186E04
:2053C200E0540275F00045F0600C901871E054081200FA1201BA45F0700302541374027565
:2053E200F000C0E0C0F012028D1581158190186EE0540275F00045F0600C901871E05408F7
:205402001200FA1201BA45F07003025413D294C29390186EE0540175F00045F060069018F2
:2054220071E054087003025457740275F000C0E0C0F012028D1581158190186EE0540175E5
:20544200F00045F06006901871E054087003025457C294D293025047121C757FFA0200D107
:20546200D294D29375C50075EB0075A80075E80075B80075F8007587007589007588007545
:20548200C80075C800758780758920758DFD758BFD75884975985212023F12026812025295
:2054A2001203E37401901876F0E475F0C0C0E0C0F0901876E075F000C0E0C0F012599A1549
:2054C2008115811581158174C875F000C0E0C0F012028D158115817405901876F0E475F0F9
:2054E200C0C0E0C0F0901876E075F000C0E0C0F012599A158115811581158174C875F000E9
:20550200C0E0C0F012028D158115817407901876F0E475F0C0C0E0C0F0901876E075F00027
:20552200C0E0C0F012599A158115811581158174C875F000C0E0C0F012028D15811581748A
:205542000F901876F0E475F0C0C0E0C0F0901876E075F000C0E0C0F012599A1581158115DA
:2055620081158174C875F000C0E0C0F012028D15811581741F901876F0E475F0C0C0E0C04A
:20558200F0901876E075F000C0E0C0F012599A158115811581158174C875F000C0E0C0F018
:2055A20012028D15811581743F901876F0E475F0C0C0E0C0F0901876E075F000C0E0C0F04F
:2055C20012599A158115811581158174C875F000C0E0C0F012028D15811581747F9018769D
:2055E200F0E475F0C0C0E0C0F0901876E075F000C0E0C0F012599A158115811581158174DC
:20560200C875F000C0E0C0F012028D1581158174FF901876F0E475F0C0C0E0C0F090187646
:20562200E075F000C0E0C0F012599A158115811581158174C875F000C0E0C0F012028D15CF
:2056420081158174FE901876F0E475F0C0C0E0C0F0901876E075F000C0E0C0F012599A158B
:205662008115811581158174C875F000C0E0C0F012028D1581158174FA901876F0E475F062
:20568200C0C0E0C0F0901876E075F000C0E0C0F012599A158115811581158174C875F00047
:2056A200C0E0C0F012028D1581158174F8901876F0E475F0C0C0E0C0F0901876E075F00095
:2056C200C0E0C0F012599A158115811581158174C875F000C0E0C0F012028D1581158174E9
:2056E200F0901876F0E475F0C0C0E0C0F0901876E075F000C0E0C0F012599A158115811558
:2057020081158174C875F000C0E0C0F012028D1581158174E0901876F0E475F0C0C0E0C0E7
:20572200F0901876E075F000C0E0C0F012599A158115811581158174C875F000C0E0C0F076
:2057420012028D1581158174C0901876F0E475F0C0C0E0C0F0901876E075F000C0E0C0F02C
:2057620012599A158115811581158174C875F000C0E0C0F012028D158115817480901876FA
:20578200F0E475F0C0C0E0C0F0901876E075F000C0E0C0F012599A1581158115811581743A
:2057A200C875F000C0E0C0F012028D15811581E4901876F0E475F0C0C0E0C0F0901876E054
:2057C20075F000C0E0C0F012599A158115811581158174C875F000C0E0C0F012028D15818D
:2057E2001581123FA2901870E054806003025838740275F000C0E0C0F012028D1581158165
:20580200901870E054806003025838901876E04480901876F0E475F0C0C0E0C0F09018767E
:20582200E075F000C0E0C0F012599A1581158115811581025835E4901876F0740175F00019
:20584200C0E0C0F0121EE6158115812223F42581F8120227125AE11202270259E4E5802254
:20586200E59022E5A022E5B022E5C022E5C422E5C822E5ED22E5EC22E5C522E5C5541060AF
:20588200FAE5C622C2AFC2AE75C5000075C50BE5C5541060FAE5C5541060F4E5C6D2AF22C7
:2058A200C2AF7F0074065388CC5389F0438901758A01758C80438810CFA295108D2040F9E4
:2058C2007E5500DEFDA296B313C2C0A295108D0E50F9D2C0CF1470E0CF030304800953886B
:2058E200EFD2C07400D2AF22C2AF7F0074065388CC5389F0438901758A01758C8043881008
:20590200CFA293108D1F50F97E2800DEFDA2C413C2C5A293108D0E40F9D2C5CF1470E1CF48
:2059220003030480095388EFD2C57400D2AF2278FB1200B68603088604741275F07A12018C
:20594200461201B1758920F58DF58B75884975985222C2AF43871075FF01D2AF22C2AF433D
:20596200871075FF01B2C6D2AF22C2AF43871075FF01B2C6D2AF2278FB1200B68682088652
:2059820083E075F0002278FB1200B68682088683E0F5F0A3E0C5F02278F91200B68682085F
:2059A200868308E6F02278F91200B6868208868308E608F0A3E6F02278FB1200B6E630991F
:2059C200FDC299F5992274FFF5F030980A3098FDC298E59975F0002278FB1200B686820824
:2059E2008683E0602D1259F3A380F778FB1200B6E63099FDC299F599B40A17740D80F2E43B
:205A020030980C3098FDC298E599B40D02740A75F0002278FB1200B6E6C0E008E6C0E012EA
:205A22005C6A13D0F0D0E0500224E02278FB1200B6E6C0E008E6C0E0125C6F13D0F0D0E0F4
:205A420050E924202278FC1200B68604188603188683188682E4FDFE125A05B4080280036C
:205A6200B47F27ED4E60F11DBDFF011E74081259F374201259F374081259F38583F0E58241
:205A82001201A785F083F58280CE1259F3F024F3600EA30DBD00010EED8EF01201C070B8D8
:205AA200E4F0ED8EF02278FB1200B68682088683E4FBFCFFE0A3B42D030FE0A3C39430B421
:205AC2000A005012FA740A75F00012012C2AFBE5F03400FC80E4EB8CF0DF030201B122127D
:205AE2005C28868208868308E4FEFFE07006125C28E4F022B42551A3E0B42D05430780A33C
:205B0200E0B4300343074024D0B40A00500BCE75F00AA42EFEA3E080EEE0B46413E60886A8
:205B2200F030F7084307201201B1A6F018F68003B4750543070A8021B478054307108019A8
:205B4200B46F104307088011125C28F0A3125C28A38095B462624307027A00C004C005C02F
:205B620006C007AB0753031F7C00E60886F0120146A6F018F6EDD007D006D005D0042430BB
:205B8200B43A0040022407C0E00AE645F070CC125C28A902EF30E505742DF0A30A125C3180
:205BA200D0E0F0A3D9FA0808EF30E7A1EAC39E509C7420F0A30A80F4B4630DAA01125C28D5
:205BC200125C31E6F0A380DEB47331C082C08386820886837A00E06004A30A80F986831852
:205BE2008682125C28125C31125C28E0A3125C286004F0A380F2D005D00480AAB4691B86BD
:205C0200017A00E76004090A80F9125C28125C318601E76091F009A380F8F97A01125C287E
:205C2200125C31E9809ECDC583CDCCC582CC22EE601A8FF020F715C002EAC39E500C7420C9
:205C420030F6027430F0A30A80EFD00222D005D006125C966009C006C00522D005D00612F4
:205C62005C6F70F2C006C00590617A802A90415A802590217E802090007F801BD005D00661
:205C8200904146125C9970CE906166125C9970C6C006C00590303978FB1200B6E6B5830035
:205CA200400EB5820975F00008E67004042240F5E42278FB1200B6E690001FB47FDF80E5E5
:205CC200D003D004125C4FC004C00370E390207E80C578FB1200B6E6C3940960C81460C52F
:205CE200C3941660C080C93200000014002003230020034B0000001E00E8032C00E80312A0
:205D0200001D00320000001400E8032300E8034B0000001E00B0042C00B00412001D0032C7
:205D220000000014004C0423004C044B0000001E0078052C00780512001D00320000001486
:205D420000B004230014054B0000001E0008072C00080712001D00370000001E0020031ED9
:205D62000020034B000000230020032000200300000C00370000001E00E8031E00E8034B8A
:205D82000000002300E8032000E80300000C00370000001E00B0041E00B0044B0000002393
:205DA20000B0042000B00400000C00370000001E0078051E0078054B0000002300780520D5
:205DC20000780500000C003C0000001E00E8032600E803500000002400E8032E00E803006A
:205DE200000C003C0000001E00B0042600B004500000002400B0042E00B00400000C003C5B
:205E02000000001E0014052600140550000000240078052E00780500000C003C0000001E08
:205E2200007805260078055A000000280040062E00400603000C00370000001200E8032899
:205E420000E803520000002500E8033000E80303000D00370000001200B0042800B004529D
:205E62000000002500B0043000B00403000D00370000001200140528001405520000002539
:205E82000078053000780503000D003700000012007805280078055200000025004006306E
:205EA20000400603000D003C0000001400E8033200E8035A0000002300E8032800D00703C8
:205EC200000D003C0000001400B0043200B0045A0000002300B0042800600903000D003CBB
:205EE20000000014007805320078055A000000230078052800F00A03000D003C00000014E4
:205F0200004006320040065A000000230040062800800C03000D00410000001900E80332C3
:205F220000E8035A0000002800E8033C00E80303001D00410000001900B0043200B0045A72
:205F42000000002800B0043C00B00403001D004100000019007805320078055A000000284B
:205F62000078053C00780503001D004100000019004006320040065A000000280040063CAD
:205F820000400603001D00460000002300200334002003640000003700E8034100E8030301
:205FA200000D00460000002300E8033400E80364000000370078054100780503000D004633
:205FC2000000002300B0043400B00464000000370008074100080703000D0046000000238D
:205FE20000780534007805640000003700D0074100D00703000D004B0000002800B0043779
:2060020000B004640001004100DC054600DC05020005004B0000002800B0043700B004649F
:206022000001004100D0074600D007020005004B00000028007805370078056400010041D7
:2060420000C4094600C409020005004B0000002800780537007805640001004100B80B4604
:2060620000B80B02000500280000000F0020031A0020034B000000180020032800200303E9
:20608200000500280000000F00E8031A00E8034B0000001800E8032800E803030005002841
:2060A2000000000F00B0041A00B0044B0000001800B0042800B00403000500280000000F1B
:2060C2000078051A0078054B000000180078052800780503000500370000001400E80332B5
:2060E2000020034B000000200078053700E80303000D00370000001400B0043200E8034BFA
:20610200000000200040063700B00403000D0037000000140078053200B0044B0000002003
:206122000008073700780503000D003700000014004006320078054B0000002000D00737D1
:2061420000400603000D00280000000F00E8031E00E8034B0000002300E8032000E8030355
:20616200000C00280000000F00B0041E00B0044B0000002300B0042000B00403000C002827
:206182000000000F0078051E0078054B000000230078052000780503000C00280000000F08
:2061A2000040061E0040064B000000230040062000400603000C00320000001000B0041EF6
:2061C20000FC084B0000001C0098082300AC0D03000C0032000000100078051E00C4094BD2
:2061E2000000001C00C4092300A00F03000C0032000000100008071E00F00A4B0000001C03
:2062020000B80B2300941103000C00320000001000D0071E00B80B4B0000001C00AC0D23A5
:2062220000881303000C00370000001200E8032300D007520000001C0040062300AC0D03F1
:20624200000C00370000001200B00423009808520000001F00D0072300A00F03000C003710
:206262000000001200780523006009520000001F0060092300941103000C00370000001207
:2062820000280A2300100E520000001F00F00A2300881303000C0000000000000000000051
:2062A2000000000000000000000000000000000000000000000000000000000000000000DC
:2062C2000000000000000000000000000000000000000000000000000000000000000000BC
:2062E20000000000000000000000000000000000000000000000000000000000000000009C
:2063020000000000000000000000000000000000000000000000000000000000000000007B
:2063220000000000000000000000000000000000000000000000000000000000000000005B
:2063420000000000000000000000000000000000000000000000000000000000000000003B
:2063620000000000000000000000000000000000000000000000000000000000000000001B
:206382000000000000000000000000000000000000000000000000000000000000000000FB
:2063A2000000000000000000000000000000000000000000000000000000000000000000DB
:2063C2000000000000000000000000000000000000000000000000000000000000000000BB
:2063E200000000000000005B32343B3448005B4B004853533E204D4138333820494E4954AC
:20640200005B32343B3448005B4B004853533E203135487A2050773D2564005B32343B340B
:2064220048005B4B004853533E203630487A2050773D2564005B32343B3448005B4B0048E5
:2064420053533E20313830487A2050773D2564005747444920414C4C41524D00454E442033
:206462005747444920414C4C41524D005747444920414C4C41524D00454E442057474449F0
:2064820020414C4C41524D005747444920414C4C41524D00454E44205747444920414C4C02
:2064A20041524D005747444920414C4C41524D00454E44205747444920414C4C41524D00FB
:2064C2005747444920414C4C41524D00454E44205747444920414C4C41524D005747444990
:2064E20020414C4C41524D00454E44205747444920414C4C41524D005747444920414C4CA2
:2065020041524D00454E44205747444920414C4C41524D005747444920414C4C41524D009A
:20652200454E44205747444920414C4C41524D005B32343B3448005B4B004853533E204DA7
:20654200792063726561746F722053746566616E6F2047414E5A455454492C207370656343
:2065620069616C207468616E6B7320746F2050494C59005B373B384800253862005B313110
:206582003B31314800253162005B31313B32334800253162005B31313B33344800253162A0
:2065A200005B31313B34354800253162005B31313B35364800253162005B373B323348009B
:2065C200253862005B31323B32334800253162005B373B33384800253862005B393B31312C
:2065E2004800253162005B393B32334800253162005B393B33344800253162005B393B342C
:20660200354800253162005B393B35364800253162005B31303B34354800253162005B311D
:20662200303B35364800253162005B31323B31314800253162005B373B35334800253862EB
:20664200005B31303B31314800253162005B31303B32334800253162005B31303B333448DD
:2066620000253162005B31313B36354800253162005B31313B37344800253162005B3132DC
:206682003B33344800253162005B31323B34354800253162005B31323B3536480025316290
:2066A200005B383B394800253162005B383B31374800253662005B383B3331480025316264
:2066C200005B383B33394800253662005B383B35334800253162005B383B3631480025366B
:2066E20062005B353B31384800253564005B31343B3230480020005B31343B32354800206D
:20670200005B31343B3330480020005B31343B323048002A005B31343B323548002A005BB3
:2067220031343B333048002A005B31363B32304800253364005B31363B3239480025316415
:20674200005B31363B33364800253364005B31363B34354800253564005B31363B353648B1
:2067620000253364005B31363B36354800253564005B31363B3735480031307546003135BA
:2067820075460032307546003235754600333075460034307546005B31373B3230480025F3
:2067A2003364005B31373B32394800253164005B31373B33364800253364005B31373B3438
:2067C200354800253564005B31373B35364800253364005B31373B36354800253564005B45
:2067E20031373B3735480032754635002035754600377546350031307546005B324A005B99
:206802004800CDCDCDCDCDCDCDCDCDCDCDCDCDCDCDCDCDCDCDCDCDCDCDCDCDCDCDCDCDCD28
:20682200CDCDCDCDCDCDCDCDCDCDCDCDCDCDCDCDCDCDCDCDCDCDCDCDCDCDCDCDCDCDCDCDB6
:20684200CDCDCDCDCDCDCDCDCDCDCDCDCDCDCDCDCD000AB0B0B0B1B1B22050756C73652022
:2068620057697468204D6F64756C6174696F6E2048494748205350454544205354415254BF
:20688200455220B2B1B1B0B0B020666F722048535320523220205B48787830312E30303709
:2068A2005D20000ACDCDCDCDCDCDCDCDCDCDCDCDCDCDCDCDCDCDCDCDCDCDCDCDCDCDCDCDE3
:2068C200CDCDCDCDCDCDCDCDCDCDCDCDCDCDCDCDCDCDCDCDCDCDCDCDCDCDCDCDCDCDCDCD16
:2068E200CDCDCDCDCDCDCDCDCDCDCDCDCDCDCDCDCDCDCD000A2020202020202020202020F5
:20690200202020202020202020202020202020202020202020202020202020202020202075
:20692200202020202020202020202020202020202020202020202020202020202020202055
:2069420020202020000AC4C420E64320535441545553206174205B20202020205D20C4C4C1
:20696200C4C4C4C4C4C4C4C4C4C4C4C4C4C4C4C4C4C4C4C4C4C4C4C4C4C4C4C4C4C4C4C495
:20698200C4C4C4C4C4C4C4C4C4C4C4C4C4C4C4C4C4C4C4C4C4000A202020202020202020B7
:2069A2002020202020202020202020202020202020202020202020202020202020202020D5
:2069C2002020202020202020202020202020202020202020202020202020202020202020B5
:2069E200202020202020000A20202050313A5B20202020202020205D202050333A5B202060
:206A02002020202020205D202050343A5B20202020202020205D202050353A5B20202020C7
:206A2200202020205D202020202020202020202020202020202020000A2020205A42313AC6
:206A42005B205D202054313A5B2020202020205D20205A42323A5B205D202054323A5B204A
:206A620020202020205D20205A42333A5B205D202054333A5B2020202020205D20202020FD
:206A82002020202020202020000A20202020205243313A5B205D20202020205243323A5B76
:206AA200205D202020205243333A5B205D202020205243343A5B205D202020205243353A1E
:206AC2005B205D20202020202020202020202020202020202020202020000A202020204949
:206AE2005354313A5B205D20202020495354323A5B205D202020495354333A5B205D202021
:206B020020205254313A5B205D202020205254323A5B205D20202020202020202020202060
:206B220020202020202020202020000A20202020205852523A5B205D2020202020584652CB
:206B42003A5B205D202020205841543A5B205D20202020594E533A5B205D202020205948F5
:206B6200533A5B205D20205848533A5B205D20205853443A5B205D20202020000A2020203E
:206B8200524F544F4B3A5B205D202057475F44574E3A5B205D202045324253593A5B205D63
:206BA20020204A4D5032333A5B205D20204A4D5032373A5B205D2020202020202020202053
:206BC200202020202020202020202020000A202020202020202020202020202020202020E9
:206BE200202020202020202020202020202020202020202020202020202020202020202093
:206C02002020202020202020202020202020202020202020202020202020202020000AC404
:206C2200C420545542452053544154555320C420312820292032282029203328202920C429
:206C4200205B202020202020202020202020202020202020202020202020202020202020F7
:206C6200202020202020202020205D20C4C4000A20202020202020202020202020202020C3
:206C82002020202020202020202020202020202020202020202020202020202020202020F2
:206CA2002020202020202020202020202020202020202020202020202020202020202000F2
:206CC2000A2020204C6F77202053706565642020504C3A5B2020205D204F4D3A5B205D20C9
:206CE200504D3A5B2020205D20544C3A5B20202020205D2050463A5B2020205D2054463A55
:206D02005B20202020205D20433A5B202020205D000A202020486967682053706565642029
:206D220020504C3A5B2020205D204F4D3A5B205D20504D3A5B2020205D20544C3A5B2020D1
:206D42002020205D2050463A5B2020205D2054463A5B20202020205D20433A5B20202020A8
:206D62005D000A20202020202020202020202020202020202020202020202020202020200A
:206D82002020202020202020202020202020202020202020202020202020202020202020F1
:206DA200202020202020202020202020202020202020000AC4C4205455424553204C494265
:206DC2005241525920C4C4C4C4C4C4C4C4C4C4C4C4C4C4C4C4C4C4C4C4C4C4C4C4C4C4C4A7
:206DE200C4C4C4C4C4C4C4C4C4C4C4C4C4C4C4C4C4C4C4C4C4C4C4C4C4C4C4C4C4C4C4C411
:206E0200C4C4C4000A202020202020202020202020202020202020202020202020202020BA
:206E2200202020202020202020202020202020202020202020202020202020202020202050
:206E42002020202020202020202020202020202020202020000A2020205B2020202020202B
:206E6200202020202020202020202020202020202020202020202020202020202020202010
:206E820020205D203C112D3E203C2D103E203C533E746F7265203C433E7573746F6D2020A8
:206EA2002020202020000A2020202020202020202020202020202020202020202020202006
:206EC2002020202020202020202020202020202020202020202020202020202020202020B0
:206EE20020202020202020202020202020202020202020202020000AC4C4C4C4C4C4C4C4A6
:206F0200C4C4C4C4C4C4C4C4C4C4C4C4C4C4C4C4C4C4C4C4C4C4C4C4C4C4C4C4C4C4C4C4EF
:206F2200C4C4C4C4C4C4C4C4C4C4204D455353414745204152454120C4C4C4C4C4C4C4C409
:206F4200C4C4C4C4C4C4C4000A2020204853533E000A706F74656E7A61206C616E63696F9C
:206F62002062617373612076656C6F63697461273A20000A706F74656E7A61206D616E7412
:206F8200656E696D656E746F2062617373612076656C6F63697461273A20000A74656D70AE
:206FA2006F206C616E63696F2062617373612076656C6F63697461273A20000A706F7465E6
:206FC2006E7A61206672656E61747572612062617373612076656C6F63697461273A20005C
:206FE2000A74656D706F206672656E617475726120666F727A6174612061207A65726F3AC6
:2070020020000A706F74656E7A61206C616E63696F20616C74612076656C6F63697461274D
:207022003A20000A736F7672616D6F64756C617A696F6E65206C616E63696F20616C7461C0
:207042002076656C6F63697461273A20000A706F74656E7A61206D616E74656E696D656EDF
:20706200746F20616C74612076656C6F63697461273A20000A74656D706F206469206C6168
:207082006E63696F20616C74612076656C6F63697461273A20000A706F74656E7A612072EE
:2070A2006964757A696F6E652076656C6F63697461273A20000A74656D706F20726964756C
:2070C2007A696F6E652076656C6F63697461273A20000A706F73697A696F6E652072656C44
:2070E20065272062617373612076656C6F63697461273A20000A706F73697A696F6E6520D6
:2071020072656C6527204B20616C74612076656C6F63697461273A20005B324A005B4800FF
:207122000AC9CDCDCDCDCDCDCDCDCDCDCDCDCDCDCDCDCDCDCDCDCDCDCDCDCDCDCDCDCDCD74
:20714200CDCDCDCDCDCDCDCDCDCDCDCDCDCDCDCDCDCDCDCDCDCDCDCDCDCDCDCDCDCDCDCD8D
:20716200CDCDCDCDCDCDCDCDCDCDCDCDCDCDCDBB000ABA20202020202020202020202020EB
:207182002020202020202020202020202020202020202020202020202020202020202020ED
:2071A2002020202020202020202020202020202020202020202020202020202020202020CD
:2071C200BA000ABA20202020202020202020202020202020202020202020434F4E464947B9
:2071E2005552415A494F4E45205455424F205649412053455249414C4520202020202020C1
:207202002020202020202020202020202020202020BA000ABA20202020202020202020206E
:2072220020202020202020202020202020202020202020202020202020202020202020204C
:2072420020202020202020202020202020202020202020202020202020202020202020202C
:207262002020BA000AC8CDCDCDCDCDCDCDCDCDCDCDCDCDCDCDCDCDCDCDCDCDCDCDCDCDCD6E
:20728200CDCDCDCDCDCDCDCDCDCDCDCDCDCDCDCDCDCDCDCDCDCDCDCDCDCDCDCDCDCDCDCD4C
:2072A200CDCDCDCDCDCDCDCDCDCDCDCDCDCDCDCDCDCDCDBC000A000A20412920706F746563
:2072C2006E7A61206C616E63696F2062617373612076656C6F63697461273A20202020202B
:2072E2002020202020202564000A20422920706F74656E7A61206D616E74656E696D656E41
:20730200746F2062617373612076656C6F63697461273A20202020202564000A20432920A7
:2073220074656D706F206C616E63696F2062617373612076656C6F63697461273A2020202E
:20734200202020202020202020202564000A20442920706F74656E7A61206672656E61740A
:207362007572612062617373612076656C6F63697461273A20202020202020202564000A2E
:207382002045292074656D706F206672656E617475726120666F727A6174612061207A6599
:2073A200726F3A20202020202020202020202564000A20462920706F74656E7A61206C6120
:2073C2006E63696F20616C74612076656C6F63697461273A202020202020202020202020E8
:2073E2002564000A20472920736F7672616D6F64756C617A696F6E65206C616E63696F3AA6
:207402002020202020202020202020202020202020202564000A20482920706F74656E7A46
:2074220061206D616E74656E696D656E746F20616C74612076656C6F63697461273A2020E0
:20744200202020202564000A2049292074656D706F206469206C616E63696F20616C7461FB
:207462002076656C6F63697461273A20202020202020202020202564000A204C2920706FAB
:2074820074656E7A6120726964757A696F6E652076656C6F63697461273A20202020202037
:2074A20020202020202020202564000A204D292074656D706F20726964757A696F6E652043
:2074C20076656C6F63697461273A202020202020202020202020202020202564000A204EF1
:2074E2002920706F73697A696F6E652072656C6527206B312C6B322C6B332C6B342C6B358C
:20750200206120363020487A3A202020253862000A204F2920706F73697A696F6E652072F3
:20752200656C6527206B312C6B322C6B332C6B342C6B3520612031383020487A3A2020254B
:157542003862000A0A20582920202020205553434952450A0070
:00000001FF
